:1000000025C043C042C041C040C03FC03EC03DC00B
:100010003CC03BC03AC039C038C037C036C08B99ED
:10002000A2ABB0B4B9BEC2FF03146EE6FFFFFFFF80
:10003000000000000007385A89FF01020305060886
:1000400009000204070900F3F4EE090011241FBEA1
:10005000CFE5D1E0DEBFCDBF20E0A0E6B0E001C03B
:100060001D92A537B207E1F7E6E7F0E0128281E0E2
:100070008683808788E58187E0E6F0E08DEF8783DF
:100080008EEF8583712C8BD028C2BACF815090E03F
:10009000FC01E85DFF4FE491E9BDFC01EF5CFF4F1F
:1000A000849188BD089520ED37E0019720F0F90193
:1000B0003197F1F7FACF089588EE93E0F4CF369AAE
:1000C0003699FECF85B10895CF93C72D81E0870D76
:1000D0008F73782E662D90E0F2D16FEF8C2F90E029
:1000E000CF91EDC1FF920F931F93CF93DF93F82E23
:1000F00007E710E0CEE7D0E0F11005C0CE01D7D180
:10010000F801808304C0F8016081CE01D8D1219725
:100110000F5F1F4FC537D10579F7DF91CF911F9141
:100120000F91FF900895D0DF81E0DCCF811103C0F3
:1001300019BC18BC0895AACF0F931F93CF93C82F53
:100140008B01CC2361F082E0A1DFC801ACDF19BCD8
:1001500018BCC801A8DFC801A6DFC150F2CFCF91FB
:100160001F910F9108951F93CF93DF938FEA87B963
:1001700086EC86B910E1C0E0D0E085E090E093DF46
:100180009EDFC80FD11D1150C1F7CE0124E0969516
:1001900087952A95E1F7DF91CF911F9108951092ED
:1001A000750083EA87B986EC86B93699FECF369A10
:1001B00086B1D82FD07486FDFBCF85B18095582E9F
:1001C000712C872D90E073D1682E8F3F31F08FEF27
:1001D00068120AC0612CA7DF09C0872D91E0970D36
:1001E000792E803470F3F3CF80E07CDF20917E00A5
:1001F0002F5F4AE350E0222391F0CA010196FC01EF
:100200003197E491AD2FB0E0A859BF4FEC93EE23A6
:1002100019F0D82FD41BF2CF2150AC01ECCFD093E2
:10022000800084E08D0F982F9150E92FED1BF0E0B6
:10023000E95BFF4FE491A92FB0E0A859BF4FEC93C1
:100240009D13F2CFE82FF0E0E959FF4F91E0309194
:1002500068002081321390E0891B80938100962DE5
:10026000953FD0F5252D2134B0F4809182008F3F49
:1002700029F4809175008093820006C081E0860D8C
:10028000682E8D1708F0612C809182008F5F8F712E
:100290008093820021C090917500909382002F3A44
:1002A000B8F490917C00992369F0962D6D1202C0EC
:1002B000612C12C0662019F09150692E0DC081503A
:1002C000682E0AC081E0860D682E8D1788F704C05D
:1002D00080917800882361F38FE384BB8BE087BB38
:1002E00088EF88BB81E083BF81EA8ABD87B986EC4D
:1002F00086B9D62DD53F10F0612C37C08091820091
:10030000803138F4E62DF0E0E859FF4FD081CD2F51
:100310002CC0D2DE8091750080938200C7E7D0E0C8
:1003200000E010E0FF24F39481E0800F0F5F1F4F87
:1003300098819F3FA9F06DE570E0FEDEF801E05A7C
:10034000FF4F608088818F258883EDDE6FE070E04D
:1003500080E2F2DE88818F258883612CE4DEACDECA
:1003600021960730110501F7CDCFAEDE10E000E099
:1003700091EAF92E26ECE22EDD24DA94DE3E81F4B9
:1003800088E0C82E89E082DE81E290E08CDE19BC34
:1003900018BC83E490E087DECA94C110F3CF47C055
:1003A000D33F41F489E072DE8AE090E07CDE85E0B4
:1003B0006DDE23C0D43F79F482DE982F80E0E82FF1
:1003C000F0E0E25EFF4FE491E91710F48F5FF7CFA2
:1003D0006DE770E010C0DE3F91F410927E00A3DE66
:1003E0006AEF70E081E0A8DE81E080937E009BDE12
:1003F0006AEF70E081E0A0DE5FDE5EDE18C0DD3F08
:1004000039F58FEF80937F008EDE82E03FDE54DE91
:1004100053DE89E03BDEA7DE80937F0084DE4CDE86
:100420004BDEF9CFC530F8F484EF91E03CDE8091EB
:1004300075008093820043DE823808F036C01F5F6B
:10044000183008F49BCFCA30A0F010E0C4E0D4E02C
:100450008C2F6CDE88DEF7B8E6B80F5F90917F00D6
:10046000891710F3DFCF0531F8F2D0927500C4E0A0
:10047000DBCFC23030F08C2F86958695C695C80F9D
:1004800013C019BC18BC85B7877E806185BFF894FE
:1004900085B7846885BF8B7F85BF85B7806285BF40
:1004A000889585B78F7D85BFDC2F10E067CFE199F8
:1004B000FECF1FBA8EBBE09A99278DB30895262FE1
:1004C000E199FECF1CBA1FBA8EBB2DBB0FB6F894B4
:0E04D000E29AE19A0FBE01960895F894FFCFCC
:00000001FF
